:100000000C9496010C94BE010C94BE010C94BE019C
:100010000C94BE010C94BE010C94BE010C94BE0164
:100020000C94BE010C9437030C9476240C94282372
:100030000C94BE010C94BE010C94BE010C94BE0144
:100040000C94540A0C94BE010C94BE010C94BE0195
:100050000C94BE010C94BE010C94BE010C94BE1A0B
:100060000C94BE010C94971F0C94DA1F0C94BE01E3
:100070000C94BE010C94BE010C94BE010C94BE0104
:100080000C94BE010C94BE010C94BE010C94BE01F4
:100090000C94BE010C94BE010C94BE010C94BE01E4
:1000A0000C94BE010C94BE010C94BE012C133213AF
:1000B00038133F134D136F138D13C71BCA1BBD1B82
:1000C000C11BEB1BEB1BEB1BCE1BD21BD61BDC1B84
:1000D000E01BEB1BE61B434C49206E6F74206176DE
:1000E00061696C61626C652C2075736520636F6E4D
:1000F000666967757261746F72210000000002000A
:10010000080E0000030401000B00000000000000C6
:100110000000000000000000000408020110408000
:1001200040102040804080080204018040201002DE
:10013000011080102040400404040404030405025C
:100140000202020403020202020606060606060472
:100150000402020204000000002300260029002CF3
:10016000002F0000000000250028002B002E003189
:100170000000000000240027002A002D00300008A5
:100180000B0002020201000904000001020200004B
:1001900005240010010524010101042402060524A0
:1001A0000600010705810310004009040100020A4E
:1001B000000000070502024000000705830240001E
:1001C0000000C18081C112010002020000404123F1
:1001D000368000010102000112010002000000400F
:1001E0004123368000010102000118034100720022
:1001F0006400750069006E006F0020004C004C0028
:1002000043002203410072006400750069006E0023
:100210006F0020004C0065006F006E0061007200EE
:1002200064006F00040309040000000000000000E7
:100230002A2B280000000000000000000000000041
:1002400000000000000000002C9EB4A0A1A2A43475
:10025000A6A7A5AE362D3738271E1F20212223241E
:100260002526B333B62EB7B89F8485868788898ABA
:100270008B8C8D8E8F909192939495969798999A56
:100280009B9C9D2F3130A3AD350405060708090A54
:100290000B0C0D0E0F101112131415161718191A36
:1002A0001B1C1DAFB1B0B500090402000103000022
:1002B00000092101010001226500070584034000B7
:1002C0000105010902A1010901A100850105091922
:1002D000012903150025019503750181029501751A
:1002E00005810305010930093109381581257F751C
:1002F0000895038106C0C005010906A10185020514
:100300000719E029E7150025017501950881029577
:1003100001750881039506750815002565050719FF
:100320000029658100C0781D4E21122611241FBEB0
:10033000CFEFDAE0DEBFCDBF12E0A0E0B1E0E0ED4C
:10034000FEE402C005900D92AA35B107D9F715E079
:10035000AAE5B2E001C01D92AC31B107E1F713E0AC
:10036000CCE2D3E004C02297FE010E94DB26C63215
:10037000D107C9F70E948A210C9466270C940000CB
:1003800080910008909101088737974709F0A89558
:100390000895DC01ED91FC910190F081E02D09952B
:1003A00008952091A0033091A103382748E0C901A6
:1003B000880F991F37FF06C09C0151E2252750E1A5
:1003C000352701C09C01415091F73093A103209340
:1003D000A003089588E38093A20380E092ECA1E05B
:1003E000B0E08093A3039093A403A093A503B093DC
:1003F000A60387E08093AF0380EC92E9ADEEB9E10C
:100400008093A7039093A803A093A903B093AA0392
:1004100085E08093B0038DEE9EEFADEABEED809354
:10042000AB039093AC03A093AD03B093AE03E1EBA9
:10043000F3E080E090E0863028F4DC01AC5DBD4F55
:100440002C9101C020E0219301968831910599F704
:1004500082E08093C9038AE08093CA03089580EC08
:1004600091EDA8E9BBE18093E7039093E803A093A3
:10047000E903B093EA0380E090E0A0E0B0E5809368
:10048000EB039093EC03A093ED03B093EE03EFEE38
:10049000F3E080E081938F5F8031E1F70895A0E081
:1004A000B0E0E5E5F2E00C94A426D82F0E94141BDE
:1004B0006115710581059105C9F30E9447271092C6
:1004C000AB031092AC031092AD031092AE03C4E0E4
:1004D000812C912C54018A94C090AB03D090AC0332
:1004E000E090AD03F090AE03FE2CED2CDC2CCC2480
:1004F0000E944227A50194010E9483266C0D7D1D58
:100500008E1D9F1D6093AB037093AC038093AD036E
:100510009093AE03C15001F7DD2309F450C001EB05
:1005200013E0E801A12CB12C62E3C62ED12CE12C02
:10053000F12C8881882309F442C0B39419F40E94F5
:10054000EA013DC00E944227A70196010E9483262E
:10055000E1E0E60FA1EBB3E08A2F801B8A1520F4BF
:100560008D918E13F9CFE9CF2091B00330E0A0E157
:10057000B7E20E941B269B01AC01AE2FB0E00E94A7
:100580002A264090A7035090A8036090A90370907A
:10059000AA03640D751D861D971D4090E7035090BA
:1005A000E8036090E9037090EA0346165706680670
:1005B000790618F2E993A39488E1A812BACFCDB7CF
:1005C000DEB7E0E10C94C02680919F03813019F4DE
:1005D00082E080939F0380919F03833019F484E02D
:1005E00080939F03089588E08093C10061E08AE0D2
:1005F0000E94EC1B60E08AE00E94251C0895009791
:10060000C9F09C0140E050E068E478EE81E090E0C1
:100610000E9483262F3F31054105510529F020F026
:100620002FEF30E040E050E02093D1008091C000F7
:10063000806103C08091C0008F7E8093C0000895C8
:10064000219A229A239860E08BE00E94EC1B61E0E3
:100650008CE00E94EC1B0895EBE6F0E0808180685E
:100660008083E8E6F0E080818160808308951F92B6
:100670000F920FB60F9211242F933F934F935F93D6
:100680006F937F938F939F93AF93BF93EF93FF935A
:100690001F9B0E94E402FF91EF91BF91AF919F9148
:1006A0008F917F916F915F914F913F912F910F901B
:1006B0000FBE0F901F901895A1E0B0E0E2E6F3E0C6
:1006C0000C94B1261FB791E090939E03F894898310
:1006D0000E94C00198E1909360008981809360003E
:1006E00081110E94C0011FBF2196E3E00C94CD262A
:1006F0008F929F92AF92BF92CF92DF92EF92FF9232
:10070000CF93FC01C0A5EC2FE770F0E0E45EFD4F55
:10071000A081B0E0C7FF03C024E130E002C02FE0B9
:1007200030E0FC0197A183E1989FF0011124E25C85
:10073000FE4F80809180A280B380A20FB31F20E47F
:100740003FE14DE750E00E943526A50194010E944B
:1007500061268C2F887149F469017A01E0EDCE0E93
:10076000E7E0DE1EE11CF11C1BC0C7FF05C060E412
:100770007AE88CE29EE004C060E07EEE8AEB9BE0CB
:1007800069017A01F8EBCF0EFBE0DF1EE11CF11CE2
:10079000A50194010E946126C20ED31EE41EF51E1F
:1007A000C701B60169517C4F8F4F9F4F28EE33E050
:1007B00040E050E00E946126A8EEB3E00E942A26A5
:1007C000CF91FF90EF90DF90CF90BF90AF909F9030
:1007D0008F9008958F3F910551F048F0811522E0E8
:1007E000920738F08115934030F482E0089580E05C
:1007F000089581E0089583E00895A0E0B0E0E3E08B
:10080000F4E00C94AD26EB018A01B82FB695A0E078
:1008100028813981F80120832A813B8121832C8121
:100820003D8122832E813F812383688179814A81A2
:100830005B812C813D81EE81FF819F2F9295990FE5
:10084000990F907C272F2370922B252F2370220F36
:10085000220F922B232F23702295207F922BF801B9
:1008600094830B5F1F4F2896AF5FBA1788F680FFFF
:1008700024C0888199810E94EA03D82E8A819B81B5
:100880000E94EA03E82E8C819D810E94EA03F82EE3
:100890008E819F810E94EA03F0E4DF9EA001112473
:1008A00090E1E99E90011124242B282BE4E0FE9E88
:1008B000B0011124262BF8012083CDB7DEB7E7E085
:1008C0000C94C926803223E0920708F1883E23E089
:1008D000920740F48F519340E4E096958795EA950E
:1008E000E1F70895803D27E0920718F48C5D93406E
:1008F0000895883928E0920768F4885C974074E08E
:10090000969587957A95E1F78D509C4F089580E0F4
:1009100090E008958FEF93E008958C30910540F4B6
:10092000A4E0880F991FAA95E1F7885D9C4F089570
:10093000843F23E0920718F484529C4F0895811558
:1009400024E0920740F48657934FF4E0880F991FF4
:10095000FA95E1F7089580E998E008959C013695AD
:10096000279525753575821B930B9C012373337373
:10097000969587959695879583739373820F931FAA
:100980009C0154E0369527955A95E1F7280F391FB9
:100990002F703F7041E051E0249FC001259F900DD2
:1009A000349F900D1124892F08952998882319F0D8
:1009B00000002A9A02C000002A980000299A00002C
:1009C0000895299A000083B12998000083FB8827A5
:1009D00080F90895CF93DF93D82F5E9A29985E9877
:1009E000C8E08D2F80780E94D504DD0FC150C9F773
:1009F0002998DF91CF9108958F770E94EA04089596
:100A0000CF93DF93D82FC8E08D2F80780E94D50434
:100A1000DD0FC150C9F72998DF91CF910895CF9389
:100A2000DF932998C8E080E0D82FDD0F0E94E10411
:100A30008D0FC150C9F7DF91CF9108950E94FC043A
:100A40000E940F055E9A0895A1E0B0E0EAE2F5E0A9
:100A50000C94B226806869830E94EA046981862F1B
:100A60000E9400055E9A2196E2E00C94CE26CF9378
:100A7000C091AB03C827E82FF0E0EE55FC4F678527
:100A800089E70E9424056C2F8DE30E9424056C2FBA
:100A900082E40E942405CF91089586E20E941E05FB
:100AA0000895CF93DF93EC016C818CE10E942405C3
:100AB0006D818DE10E9424056E818EE10E942405E6
:100AC0006F8180E20E942405688581E20E942405EE
:100AD000698582E20E9424056A8583E20E942405DA
:100AE0006B8584E20E9424056C8585E20E942405C2
:100AF0006D858AE20E9424056E858EE60E9424059B
:100B00006F858FE60E942405688980E70E9424058E
:100B1000698981E70E9424056A8982E70E94240589
:100B2000DF91CF910895CF92DF92EF92FF92CF9312
:100B3000DF936B017C01C11488E3D8068CE9E806D9
:100B40008CE1F80628F5C701B60120E836E948E946
:100B500050E00E946126E901689760E879E687E63F
:100B60009FEF0E943D266C0D7D1D8E1D9F1DF2E0A6
:100B7000660F771F881F991FFA95D1F721E732E09A
:100B800040E050E00E946126F22EE32E80E421C076
:100B9000C701B60120E03DE241E351E00E94612639
:100BA000E901689760E073ED8EEC9EEF0E943D26B0
:100BB0006C0D7D1D8E1D9F1D660F771F881F991F51
:100BC00021E732E040E050E00E946126F22EE32E61
:100BD00080E66C2F6F71680F85E70E9424056E2DEB
:100BE00086E70E9424056F2D87E70E942405DF9188
:100BF000CF91FF90EF90DF90CF900895682F8DE612
:100C00000E94240508958F929F92AF92BF92CF9237
:100C1000DF92EF92FF92CF93DF93D82F83E00E9471
:100C20001E0580939D0384E00E941E0580939C0313
:100C300060E086E00E94240561E087E00E942405D0
:100C40006FE789E00E94240565E08AE00E942405A0
:100C500065E18BE00E94240562E18CE00E9424059E
:100C60006DEF8DE00E94240560E08EE00E94240577
:100C7000DD2319F08BE291E008C02091C90333E134
:100C8000239FC0011124825C9E4F0E9451056CE895
:100C900080E30E9424056FE082E30E94240562E461
:100CA00083E30E9424058091CA0387FF02C064E1A8
:100CB00001C06AE084E30E9424056AE285E30E94A1
:100CC00024056DE286E30E94240564ED87E30E941B
:100CD000240560E088E30E94240560E089E30E9427
:100CE0002405D11109C0C090AB03D090AC03E090B3
:100CF000AD03F090AE0307C0C5E9CC2EC1ECDC2EED
:100D0000ED2CCEEDFC2ECAE38F2C9924AA24BB2413
:100D1000682D8C2F0E942405682D85E08C0F0E9481
:100D20002405FE2CED2CDC2CCC24CF5FCE3361F7D8
:100D30006FEF83E40E9424056FEF84E40E94240592
:100D40006FEF85E40E9424056FEF86E40E9424057E
:100D5000DD2311F066E002C06091AF038DE60E94D2
:100D6000240560E089E70E9424056091B0038AE7CA
:100D70000E94240560E083E70E94240560E084E788
:100D80000E942405D11109C06091A7037091A803A6
:100D90008091A9039091AA0304C060EC72E98DEEE2
:100DA00099E10E949305DF91CF91FF90EF90DF9042
:100DB000CF90BF90AF909F908F90089561E087E0B3
:100DC0000E94240564E28EE70E94240563E088E027
:100DD0000E94240560E088E00E94240565E087E029
:100DE0000E94240562E085E00E94240583E00E94C1
:100DF0001E0580939D0384E00E941E0580939C0342
:100E0000089583E00E941E0580939D0384E00E9464
:100E10001E0580939C0361E087E00E9424056AE040
:100E200070E080E090E00E94371B0E94DE06000028
:100E30000895CF92DF92FF920F931F93CF93DF938A
:100E40001F92CDB7DEB7082F162F8EE399830E942D
:100E50002405F02EC02E9981D92E8C2D8F19811743
:100E600038F4F60161916F018FE70E942405F5CFF8
:100E700064E085E00E94240583E00E941E058093C3
:100E80009D0384E00E941E0580939C030E94141B16
:100E9000609398037093990380939A0390939B03B4
:100EA00069E087E00E94240581E080939F030F9012
:100EB000DF91CF911F910F91FF90DF90CF90089518
:100EC0000F931F930E94190780919F03813099F41B
:100ED0000E94141B009198031091990320919A038A
:100EE00030919B03601B710B820B930B603A764829
:100EF0008140910548F380919F03813031F467EA86
:100F000071E08AE094E00E941C1E1F910F910895E9
:100F10000F931F9380919F03823021F410929F03BF
:100F200081E020C080919F038130D9F40E94141B7E
:100F3000009198031091990320919A0330919B039B
:100F4000601B710B820B930B613A764881409105CF
:100F500040F061E087E00E94240510929F0382E048
:100F600001C080E01F910F910895CF93DF93EC01B2
:100F70004AE050E06D2F70E08AE094E00E94E11EAC
:100F80006EE28AE094E00E94EE1DBE0184E0769558
:100F900067958A95E1F76F7077274AE050E08AE01D
:100FA00094E00E94E11E6EE28AE094E00E94EE1D51
:100FB000BE016F7077274AE050E08AE094E00E941B
:100FC000E11EDF91CF910895D82FC0E0CD1780F4B6
:100FD0005F9A64E670E080E090E00E94371B5F98C3
:100FE00064E670E080E090E00E94371BCF5FEECFB8
:100FF0006CE271E080E090E00E94371BE6CF0F9337
:101000001F93CF93DF93EC01062F15E0115051F0A1
:10101000CE010E945027081741F0602FCE010E9498
:101020005827F4CF82E00E94E407DF91CF911F910F
:101030000F910895A0E0B0E0E0E2F8E00C94A4265F
:10104000482E562EC0E0D0E0612C712CE12CF12C02
:1010500000E010E041100CC06090000486E4689E3F
:101060003001112459E1E52EF12C06EE13E01EC0EB
:1010700091E049120FC060900004E6E46E9E3001DA
:101080001124FBE16F0E711C49E2E42EF12C02EAFF
:1010900013E00CC082E0481209C028E1622E7724D8
:1010A0007394EE24E394F12C0FEF13E043018C0EC4
:1010B0009D1E1092A1031092A0033401A62CA81823
:1010C000B12CC30101966C01AE14BF04A8F4A00EAC
:1010D000B11E511006C0C3010E945027F501808344
:1010E00005C0F5016081C3010E94FF07F501808101
:1010F0000E94D1013601E2CFC301511018C0C301D3
:101100000E945027B82EC6010E9450272B2D30E098
:10111000322F2227282B8091A0039091A1038217C0
:10112000930779F4C0E0D0E05524539493CF36016F
:101130006091A1030E94FF076091A003C6010E9475
:10114000FF07C05EDE4FC13E92E0D90708F482CFB0
:10115000852DCDB7DEB7E0E10C94C02661E082E0DA
:101160000E941A08089560E082E00E941A088091A7
:10117000FF03853020F01092FF030E94AE0880919B
:10118000FF0380930004089561E080E00E941A0844
:1011900061E081E00E941A08089560E080E00E940A
:1011A0001A08882351F060E081E00E941A08882321
:1011B00021F08091A203883349F00E942F020E94FF
:1011C000EA0181E00E944F020E94C4080895CF9373
:1011D000C82F0E94141B60935C0370935D0380937F
:1011E0005E0390935F03C0937103CC2329F040E02A
:1011F00051EE60E070E004C040E855E260E070E06D
:101200008CE594E00E944720CF910895909160036F
:10121000492F4F7050E0BA016F5F7F4F292F30E0A8
:10122000E4E035952795EA95E1F76217730759F0E1
:10123000FA01EF59FC4F808381E0890F8F70907F16
:10124000892B8093600308956EE770E08CE594E04D
:101250000E94C9010895A3E1B1E0E1E3F9E00C9433
:10126000A526E1EBF3E0712C8191882321F07394A2
:1012700028E17212F9CF63EB71E08AE094E00E94FA
:101280001C1E4AE050E0672D8AE094E00E94E81EB0
:1012900080E00E9403060E94DE068E010E5F1F4F53
:1012A000C12CD12C7601C39466246A945C2C0E94D4
:1012B000081B4B015C012091B00330E0A0E1B7E2D4
:1012C0000E941B269B01AC01C701B6010E943D266E
:1012D0002091A7033091A8034091A9035091AA033C
:1012E000620F731F841F951F2091E7033091E8035D
:1012F0004091E9035091EA03261737074807590739
:1013000018F4F801608225C08C2D0E94370561E039
:1013100070E080E090E00E94371BF80110820E948C
:10132000081B681979098A099B09643F7140810586
:10133000910540F40E944D05F8019081981778F7C7
:101340008083EDCF50FE03C046985F9A02C0469A54
:101350005F982FEFC21AD20AE20AF20A0F5F1F4FFC
:101360008FEFC816D104E104F10409F09FCFCE013C
:101370009395FC01D82E7FEF68EC2E2F281B2715A4
:1013800010F051E056C0DE01129651E02FEF41E01F
:101390003D91321710F0322F01C0452F5F5F5F3F44
:1013A00011F0232FF5CF4193242F30E0A1E0B0E0DE
:1013B000AC0FBD1FA20FB31F5C93413079F0DE016B
:1013C000A20FB31F5C93423049F0AFEFBFEFAC0FF9
:1013D000BD1FA20FB31F6C934E3F78F6A2E0B0E0A2
:1013E000AC0FBD1FA20FB31F7C934D3F30F6A3E09F
:1013F000B0E0AC0FBD1FA20FB31F6C93BECF452F43
:10140000242F30E0FC01E20FF31F6081AFEFB0E06A
:10141000AC0FBD1FA20FB31F2C91621748F44150AF
:10142000DC01A40FB11D2C9120836C934111E8CFF6
:101430005F5F571520F3372D369520E0231770F4A2
:10144000DC01A20FB11D4C91522F530FFC01E50F8F
:10145000F11D50815C9340832E5FF0CFF1EBEF2EB6
:10146000F3E0FF2E8C01802F8D19871598F4F80179
:10147000C1908F014AE050E06C2D8AE094E00E9418
:10148000D91E6CE28AE094E00E94EE1DF701C19241
:101490007F01E9CF8AE094E00E94F61D81E0CD5EF5
:1014A000DE4FEFE00C94C1261F920F920FB60F9201
:1014B00011241F932F933F934F935F936F937F93C9
:1014C0008F939F93AF93BF93CF93DF93EF93FF934C
:1014D000C0918600D09187008091170390911803E6
:1014E00020913903211155C09E01281B390B809191
:1014F000EB039091EC03A091ED03B091EE0385FD19
:1015000002C036952795253C49E03407B8F1409153
:101510000A0150E060E070E02CE1B695A795979540
:1015200087952A95D1F70097A105B10521F481E0AF
:1015300090E0A0E0B0E084179507A607B707D8F4BD
:1015400080910A018F3FB9F040E080910A0148176D
:1015500080F4842F90E0880F991FFC01E75EFC4F18
:1015600020813181FC01E55FFE4F318320834F5F95
:10157000ECCF10923A0310920A010BC02D3B82E08F
:10158000380720F080910A018031D8F08FEF8093E6
:101590000A01D0931803C0931703FF91EF91DF91D5
:1015A000CF91BF91AF919F918F917F916F915F91FB
:1015B0004F913F912F911F910F900FBE0F901F9051
:1015C000189510910A0181E0810F80930A01C901E9
:1015D0000E946204E12FF0E0EE0FFF1FE75EFC4F78
:1015E00091838083D6CF83E0809380008AE98093C3
:1015F00081008091EB0386FD05C0809181008064AD
:10160000809381008FEF9FEF9093890080938800F3
:1016100080916F00806280936F000895CF93DF9375
:101620000E94B30880910004843039F582E00E9462
:10163000581CC1E0D0E0892B11F4C0E0D0E083E079
:101640000E94581C892B19F082E090E002C080E0D3
:1016500090E08C2B9D2B8230910539F083309105E1
:1016600039F0019739F481E006C01092000405C0FA
:1016700082E001C083E080930004DF91CF91089560
:101680006F3018F086958058089589E0689F802D06
:1016900011240895A0E0B0E0E0E5FBE00C94AC2656
:1016A000C82F0E94141B0091C8021091C9022091FA
:1016B000CA023091CB026B017C01C01AD10AE20A46
:1016C000F30A9701860149E8C41643E1D406E10410
:1016D000F10410F01092CC026093C8027093C9021A
:1016E0008093CA029093CB02209139038FEF820F2F
:1016F0008230E8F5E091CC02EE2309F46EC1E130CE
:1017000011F482E0D8C1E03178F581E08E0F80934A
:10171000CC02F0E0E75EFC4FC083803109F0D4C119
:10172000EBE1F3E0213029F4A181A695A695808113
:1017300008C080819181A92FA695A695A69596951A
:101740008795A03148F4B0E090E0AA0FBB1FA55FD9
:10175000BE4F11969C938E9310923A03329683E07B
:10176000E932F807F9F6B0C11092CC02ADC12330CE
:1017700009F023C1E091CC02E11118C0CF3009F08B
:1017800011C10E94081B009147031091480320914A
:10179000490330914A03601B710B820B930B62303B
:1017A00071058105910508F089C1FCC0E83148F454
:1017B00081E08E0F8093CC02F0E0E85EFC4FC083A6
:1017C000F1C0E83109F0ECC0C111EAC040E050E0DE
:1017D000ABE0CA01B3E0880F991FBA95E1F7A49F67
:1017E0009001A59F300D1124F901E75EFC4F608147
:1017F000E1817E2F777075956795FC01EE0FFF1FD5
:10180000E55FFE4F71836083F901E65EFC4FB081B6
:10181000B695B695B695E181FE2FF295FF0FF07E55
:101820006F2F6B2BE695E695E6957E2F7770759575
:101830006795FC01EE0FFF1FE35FFE4F718360832E
:10184000F901E55EFC4FB081B295B695B695B370DF
:10185000C181DC2FDD0FDD0F6D2F6B2BC295C6957F
:10186000C695C370E281E170EE0FEE0F7E2F7C2BE8
:1018700075956795FC01EE0FFF1FE15FFE4F7183C9
:101880006083F901E35EFC4FB081B695E181FE2FE4
:10189000F795FF27F7956F2F6B2BE6957E2F7770C7
:1018A00075956795FC01EE0FFF1FEF5EFE4F71838C
:1018B0006083F901E25EFC4FB081B295BF70E181B7
:1018C000FE2FF295F07F6F2F6B2BE295EF707E2F3E
:1018D000777075956795FC01EE0FFF1FED5EFE4F6B
:1018E00071836083F901E15EFC4FB081BB1FBB27B0
:1018F000BB1FC181DC2FDD0F6D2F6B2BCC1FCC27C5
:10190000CC1FE281E370EE0F7E2F7C2B75956795DF
:10191000FC01EE0FFF1FEB5EFE4F71836083F90148
:10192000EF5DFC4FB081B695B695E181FE2FF29543
:10193000FF0FFF0FF07C6F2F6B2BE695E6957E2F48
:10194000777075956795FC01EE0FFF1FE95EFE4FFE
:1019500071836083F901EE5DFC4F2081229526950D
:1019600027703181E32FEE0FEE0FEE0F6E2F622BFB
:10197000732F72957695777075956795FC01EE0FCC
:10198000FF1FE75EFE4F718360834F5F5F4F423002
:10199000510509F01ECF80912F0383FF10923A0367
:1019A0001092CC020E94081B609347037093480377
:1019B0008093490390934A0387C0243009F084C080
:1019C0006091CC0261110BC0C83AB1F41092A1032E
:1019D0001092A00388EA0E94D10181E06CC06130BE
:1019E00019F4C093C70204C0623031F4C093C60238
:1019F0008C2F0E94D1015AC0E091C6022E2F30E0F8
:101A0000220F331F462F50E0C90102968417950715
:101A10003CF0633268F7FA01EA5EFC4FC083E8CF1E
:101A20002D5F3F4F8C2F90E06091A0037091A10338
:101A30004217530749F4982F8827862797279093B2
:101A4000A1038093A00332C06817790769F58091DC
:101A5000C702813049F5E13118F080E18093C60278
:101A6000F090C602CAE1D3E000E010E00F15D0F418
:101A7000FE013197808190E0982F88272881822B62
:101A800063E0969587956A95E1F70E946204F801F4
:101A9000EE0FFF1FE55FFE4F918380830F5F1F4FA7
:101AA0002296E4CF10923A031092CC028091CC029D
:101AB000882351F08F5F8093CC0206C08091CC02C6
:101AC0008F5F8093CC026ECFCDB7DEB7E8E00C9489
:101AD000C826CF93DF93E82FF0E0EA51FC4FE18571
:101AE000E03150F4F894F0E0EE0FFF1FE55FFE4F99
:101AF0008081918178945FC08EE08E0F8B3058F496
:101B0000F0E0E25FF10924E62E9FC0012F9F900DC7
:101B100011240C9650C0E03F09F448C038F4E1317C
:101B2000A1F0E231A1F0E03139F409C0ED3FC1F19B
:101B3000EE3FC9F1E13F89F180E092E03CC082E0F4
:101B40000E94581C892B19F134C083E0F9CF82E040
:101B50000E94581CC1E0D0E0892B11F4C0E0D0E015
:101B600083E00E94581C892B19F082E090E002C0AB
:101B700080E090E08C2B9D2B8230910541F08330EA
:101B8000910541F00197A9F086EA92E014C08CE03B
:101B900090E011C089E591E00EC086E090E00BC0B6
:101BA0008AEF93E008C08FEF93E005C080E090E0FB
:101BB00002C084EF93E0DF91CF910895A2E2B0E0FC
:101BC000E4EEFDE00C94A2269E012F5F3F4F80E1E2
:101BD000D9011D928A95E9F761EE71E08AE094E0FF
:101BE00029A33AA30E941C1E0E9401071D8A1E8A77
:101BF0001F8A188E312C212C00E0812C912C54014D
:101C000070E4472E71EE572E7DE9672E78E1772E2E
:101C1000E0E5CE2EE3ECDE2EE12CF12C84EF91E01A
:101C2000A0E0B0E08D8F9E8FAF8FB8A380EC91EDD8
:101C3000A8E9BBE1898F9A8FAB8FBC8F80E491EECE
:101C4000ADE9B8E1898B9A8BAB8BBC8B8AE094E0D1
:101C50000E94811C892B09F4E1C08AE094E00E9473
:101C6000A51C9C0133272C32310509F442C0ACF489
:101C70002332310509F0ABC019821A821B821C8203
:101C80001D821E821F82188619861A861B861C8654
:101C90001D861E861F86188A60C02434310529F0EF
:101CA0002335310509F4B2C092C064E48AE094E0BF
:101CB0000E94EE1D2AE030E040E451EE6DE978E14B
:101CC0008AE094E00E947C1E6CE28AE094E00E942C
:101CD000EE1D2AE030E040EC51ED68E97BE18AE05E
:101CE00094E00E947C1E6CE28AE094E00E942E1E2A
:101CF000ADCF0F5F043009F0A9CF29813A814B8124
:101D00005C81A8EEB3E00E942A26698B7A8B8B8BCC
:101D10009C8B2D813E814F8158850E942A26698F98
:101D20007A8F8B8F9C8F29853A854B855C852D8F8B
:101D30003E8F4F8F58A32D853E854F8558890E9431
:101D40002A266B017C0160323EE473078105910510
:101D500030F462E38CE10E94240500E077CF603329
:101D600045E774078105910510F462E2F3CF603412
:101D70005CE975078105910510F466E2EBCF80E51B
:101D8000C81683ECD806E104F10410F462E1E2CF56
:101D900090E6C9169AEED906E104F10410F465E163
:101DA000D9CFA0E7CA16A1E1DA06A1E0EA06F1045C
:101DB00010F461E0CFCFB0EACB16B6E8DB06B1E0B5
:101DC000EB06F10410F463E0C5CF65E0C3CF10ED7E
:101DD000180F1A3008F03ACFE1E0F0E0EC0FFD1FE9
:101DE00024E0029FE00DF11D112420813181428108
:101DF0005381AAE0B0E00E942A26610F711D811D67
:101E0000911D608371838283938320CF49885A8890
:101E10006B887C88812C912C540118CF81149104FB
:101E2000A104B10489F4C301B2010E94930561E0E9
:101E300070E080E090E00E94371B1D8A1E8A1F8A96
:101E4000188E312C22242A948D8D9E8DAF8DB8A1B1
:101E500088169906AA06BB06D0F40E944D052D8966
:101E60003E894F89588D280F311D411D511D2D8BE5
:101E70003E8B4F8B588F381608F4382E821508F495
:101E8000282E3FEF831A930AA30AB30A56C0C30150
:101E9000B20128EE33E040E050E00E946126BA0132
:101EA000A9012AE030E08AE094E00E94CA1E6CE2B8
:101EB0008AE094E00E94EE1D4AE050E0632D8AE043
:101EC00094E00E94D91E6CE28AE094E00E94EE1D2C
:101ED0006D897E898F89988DA50194010E94612664
:101EE000BA01A9012AE030E08AE094E00E94CA1E0B
:101EF0006CE28AE094E00E94EE1D4AE050E0622D20
:101F00008AE094E00E94D91E6CE28AE094E00E948C
:101F10002E1E4C0C5D1C6E1C7F1C898D9A8DAB8D0A
:101F2000BC8D84159505A605B70520F449885A8807
:101F30006B887C88812C912C540129893A894B89A2
:101F40005C89283E33404105510509F07FCEA296B9
:101F5000E2E10C94BE26ACE1B0E0E1EBFFE00C94D2
:101F6000AC260E94141B6B017C0181E00E940306D9
:101F700014E703E0198361E0CE0101960E94600737
:101F800000939F030E94DE066AEF70E080E090E01D
:101F90000E94371B80919F03833089F48AE094E08C
:101FA0000E94811C892B59F40E94141B6C197D0915
:101FB0008E099F096038734C894C9140D8F280910A
:101FC0009F03833009F44FC08FE70E94FC040E94F6
:101FD0000F058983843511F083E05CC00E940F05F2
:101FE00010927203809373030E940F052091720375
:101FF00030917303280F311D3093730320937203C4
:102000000E940F05809374030E940F05809375034F
:10201000813110F7F12C0F2D10E08091750390E0C5
:10202000880F991F0817190740F40E940F05F8013F
:10203000EA58FC4F8083F394EECF80E7898361E018
:10204000CE0101960E94600783E080939F030E9467
:10205000DE0662E370E080E090E00E94371B809132
:102060009F03833011F482E015C08FE70E94FC04C7
:102070000E940F058983803509F0AECF0BEC13E089
:102080000E940F05F80181938F01F3E0063E1F07C0
:10209000B9F781E06C96E8E00C94C826CF93C82F7E
:1020A000682F8AE094E00E94F21C909196039C278E
:1020B00090939603CF910895A1E0B0E0E2E6F0E1BD
:1020C0000C94B22699830E944E109981892F0E9408
:1020D0004E102196E2E00C94CE261F93CF93DF930F
:1020E000182FEB011092960365EB8AE094E00E94B2
:1020F000F21C62E68AE094E00E94F21C812F0E94AA
:102100004E10CE010E945C10DF91CF911F91089577
:10211000609196038AE094E00E94F21C0895A1E287
:10212000B0E0E5E9F0E10C94AE267B018A018C3049
:1021300009F452C108F040C0863009F4BCC018F55B
:10214000833009F491C070F4813009F472C0823098
:1021500009F049C26BE170E082E00E946D100BEC67
:1021600013E078C0843009F487C0853009F03BC2A1
:102170006091750370E0660F771F85E00E946D1017
:1021800006E713E086C0893009F4A7C070F48730F1
:1021900009F49BC0883009F026C261E070E088E055
:1021A0000E946D108091000424C28A3009F4CAC0D4
:1021B0008B3009F4F1C017C28A3609F474C1D8F41F
:1021C000873609F439C138F4853609F40DC18636ED
:1021D00009F41EC108C2883609F436C1893609F0EF
:1021E00002C261E070E089E60E946D100E94EA017F
:1021F0000E942F02F6C18D3609F4D3C138F48B3614
:1022000009F490C18C3609F499C1EDC18E3609F4F8
:10221000DDC1873C09F0E7C161E070E087EC0E9416
:102220006D1081E00E944E100E948810109297035A
:10223000E4C169E270E081E00E946D1002EA13E0FF
:10224000F80181918F010E944E10F3E00B3C1F07B3
:10225000B9F7D1C1F80181918F010E944E10F3E0CE
:10226000063E1F07B9F7C7C161E070E083E00E9436
:102270006D100E94AB0FBDC161E070E084E00E9470
:102280006D1081E00E944E100E9488100E94DE0DA9
:10229000B4C18091750390E0880F991F980126576B
:1022A00033402817390708F0A6C1F80181918F0142
:1022B0000E944E10EECF62E070E086E00E946D104A
:1022C00088E893E00E945C1096C161E070E087E0CE
:1022D0000E946D10809174038CC186E6898361E051
:1022E000CE0101960E9460070E94DE0683E0809383
:1022F0009F0368EC70E080E090E00E94371B8091C3
:102300009F038430D9F48FE70E94FC040E940F05DC
:102310008983863469F460E270E089E00E946D1080
:1023200010E20E940F050E944E101150D1F763C1B8
:1023300061E070E089E00E946D1053C161E070E0DF
:1023400089E054C169E170E08AE00E946D1010924A
:10235000E60320919E038091EB039091EC03A09102
:10236000ED03B091EE03222311F0806801C08F7756
:102370008093EB039093EC03A093ED03B093EE03F3
:1023800006EE13E0F80181918F010E944E10F3E0F8
:102390000F3F1F07B9F72FC161E270E08BE00E9489
:1023A0006D1080913A038F3F39F080913A0391E0AC
:1023B000980F90933A0302C080913A030E944E1006
:1023C00010E0812F0E94690D0E948D040E945C1014
:1023D0001F5F1031B1F70FC161E070E08CE00E9427
:1023E0006D108091FF0305C161E070E085E60E94F9
:1023F0006D1089E2E816F10409F0FAC0D801E2EAAA
:10240000F3E08D91819383E0EB3CF807D1F7E9C0CD
:1024100061E070E086E60E946D10EBE1EE16F104DB
:1024200009F0E6C0D801EBECF3E08D91819383E0F5
:10243000E63EF807D1F7D5C061E070E087E60E947C
:102440006D100E94C408CDC061E070E088E60E9473
:102450006D1085E789838BE1EBECF3E0DE011296EA
:1024600001900D928A95E1F76CE1CE0101960E94F0
:1024700060070E94DE0683E080939F0360E273E0C2
:1024800080E090E00E94371B80919F03843009F028
:10249000AFC08FE70E94FC040E940F058983853539
:1024A00009F0A6C09EC061E070E08AE60E946D104F
:1024B00089E6898361E0CE0101960E9460070E944F
:1024C000DE0683E080939F0360E273E080E090E0AB
:1024D0000E94371B80919F03843009F089C08FE7E9
:1024E0000E94FC040E940F0589838E010E5F1F4F1E
:1024F0007E01EDE1EE0EF11C0E940F05F8018193C3
:102500008F01EE15FF05C1F78BE1FE013296ABECB2
:10251000B3E001900D928A95E1F78981893409F041
:1025200067C05FC061E070E08BE60E946D10F8014B
:102530008081809300040E94CD0853C061E070E068
:102540008CE60E946D10F0E2EF16F10461F487E66C
:10255000898380E2F801DE01129601900D928A953E
:10256000E1F761E203C087E4898361E0CE0101966F
:102570000E9460070E94DE0683E080939F036CE464
:1025800074E080E090E00E94371B80919F038430CC
:1025900079F58FE70E94FC040E940F05873441F50E
:1025A00020C061E070E08DE60E946D1089E1E816C0
:1025B000F104F1F4D801E6EEF3E08D91819383E02C
:1025C000EF3FF807D1F70E94F30A0BC061E070E01B
:1025D0008EE60E946D10F80180818093FF030E94B7
:1025E000AE0881E006C061E070E08AEC0E946D10E8
:1025F00080E00E944E100E948810A196E6E00C94A4
:10260000CA26A0E0B0E0E7E0F3E10C94AC26CAE50E
:10261000D2E014E606E035E0F32E44E0E42E53E089
:10262000D52E62E0C62E8AE094E00E94811C892BA0
:1026300009F49BC08AE094E00E94A51C282F809397
:10264000C5024091C40250E04730510560F7FA01DD
:10265000EA5AFF4F0C94D926853B29F781E08093F5
:10266000C402E1CF823609F07DC0C092C402DBCF44
:102670008093C3028093C202D092C402D4CF9C0143
:1026800033273093C1022093C0029091C202982751
:102690009093C202E092C402C6CF382F2227409105
:1026A000C0025091C102242B352B3093C1022093DC
:1026B000C0029091C20298279093C202F092C40285
:1026C0002536310508F4AFCF61E070E08CEC0E9454
:1026D0006D1081E00E944E100E94881043C020912E
:1026E000BE023091BF02F901E65AFD4F80839091FE
:1026F000C20298279093C202C90101969093BF022B
:102700008093BE022091C0023091C10282179307CC
:1027100008F489CF0093C40286CF8091C20282134D
:102720000BC06091BE027091BF024AE552E08091F9
:10273000C3020E948F100DC062E070E08BEC0E941B
:102740006D108091C3020E944E10809196030E94EA
:102750004E10FE01812F11928A95E9F71092BF0267
:102760001092BE021092C4025ECFCDB7DEB7E8E091
:102770000C94C82681E08093970380919703882367
:1027800049F08AE094E00E94811C892BB1F30E94F9
:102790000113F3CF0895AAE2B0E0E1EDF3E10C9468
:1027A000AA260E94081B6B017C0181E00E9403069F
:1027B0008AE094E00E94811C892B29F08AE094E051
:1027C0000E94A51CF5CF5F9811E072E6B72EE9E2F2
:1027D000AE2E03E00E94081B6C197D098E099F092B
:1027E000693C710581059105D0F11123C1F10E9469
:1027F000081B6B017C01469A80ED97E00E94FF0266
:10280000B982E2EAF3E0DE0112968A2D01900D9280
:102810008A95E1F76AE2CE0101960E946007469828
:1028200080E090E00E94FF0200939F030E94DE067A
:1028300062E370E080E090E00E94371B80919F038C
:10284000843061F400939F038FE70E94FC040E9490
:102850000F0511E0823419F410E001C011E082E1AB
:102860000E94581C892B81F411E00EC05F9A469A91
:102870008AE094E00E94A51C8D309105A9F05CF4DB
:102880000A9791F05F9846988AE094E00E94811C34
:10289000892B61F79FCF8332910569F082349105CE
:1028A00089F70E94BA13EECF66ED70E08AE094E0FB
:1028B0000E940A1EE7CF0E94DE0DE4CF8F929F9206
:1028C000AF92BF92CF92DF92EF92FF921F93CF937E
:1028D000DF9382E10E94581C892B09F089C068ECC3
:1028E00070E080E090E00E94371B80E090E00E9462
:1028F000FF020E94081B4B015C016B017C0180EC14
:10290000C80E82E1D81EE11CF11C0E94081B6C1548
:102910007D058E059F0530F482E10E94581C892BAD
:10292000A1F364C082E10E94581C892B09F05EC0AB
:1029300080ED97E00E94FF020E94081B6B017C0162
:10294000D0E0C1E088E4880E86E2981EA11CB11C8C
:1029500011E082E10E94581C892B21F58C149D0402
:10296000AE04BF0430F480ED97E00E94FF02D1E096
:10297000F0CF0E94081B6C197D098E099F09693CE4
:1029800071058105910528F30E94081B6B017C01EC
:10299000C12719F080ED97E002C080E090E00E942E
:1029A000FF02D7CF80E090E00E94FF02DD23B9F064
:1029B0008091FF0390E0019665E070E00E944D2653
:1029C0008093FF030E94AE080E940E0B0E94CD0868
:1029D00064EF71E080E090E00E94371B09C080E066
:1029E0000E944F020E942B090E94C4080E94CB1330
:1029F000DF91CF911F91FF90EF90DF90CF90BF902C
:102A0000AF909F908F900895CF92DF92EF92FF92B8
:102A100080E00E945C030E94200361E086E00E9447
:102A2000EC1B61E085E00E94EC1B60E082E10E940B
:102A3000EC1B60E082E00E94EC1B61E082E00E94FF
:102A4000251C60E083E00E94EC1B61E083E00E94B3
:102A5000251C60E084E00E94EC1B61E084E00E94A1
:102A6000251C0E94F30260E070E08AE094E00E947E
:102A7000771D0E940E0B0E94CD080E94F30A8FEF73
:102A800080933A030E942C0378940E94081B6B01E8
:102A90007C0180913A038F3F59F40E94081B6C1906
:102AA0007D098E099F09603D77408105910588F376
:102AB00080ED97E00E94FF0261E082E10E94251C08
:102AC0005F9A8AE094E00E94811C892B29F08AE0B9
:102AD00094E00E94A51CF5CF6EEE71E08AE094E0D0
:102AE0000E94EB1D88E893E00E94B50765E072E064
:102AF0008AE094E00E94EB1D4AE050E066E070E05E
:102B00008AE094E00E94B21E62E370E080E090E010
:102B10000E94371B8AE094E00E94811C04970CF10C
:102B20008AE094E00E94A51C82349105D1F48AE0E9
:102B300094E00E94A51C8E34910599F48AE094E0FB
:102B40000E94A51C8434910561F48AE094E00E94FF
:102B5000A51C819731F480E090E00E94FF020E9462
:102B6000CB134091A3035091A4036091A5037091EE
:102B7000A603DB01CA010197A109B1090497A105C8
:102B8000B10590F440933903433051F42EE240EA0A
:102B900056E861E070E08CE594E00E94C82008C02F
:102BA00040E052EC61E070E08CE594E00E94472048
:102BB0000E945E145F9880E090E00E94FF020E94F5
:102BC000F30A109259038091EB0383FF11C08091A7
:102BD000B703882351F08091BE03882331F08091A0
:102BE000C503882311F087E001C085E08093590375
:102BF00080E00E94030680915A030E9437050E94DC
:102C0000DE061092CF021092CE021092CD02F12C6D
:102C1000809100048F15B0F062E370E080E090E0F6
:102C20000E94371B80ED97E00E94FF0262E370E094
:102C300080E090E00E94371B80E090E00E94FF025D
:102C4000F394E6CF8091CA0384FF08C0982F98714F
:102C500081E0983109F080E00E94E7088FE00E944F
:102C60005C03FF90EF90DF90CF900895EF92FF927A
:102C70000F931F93CF93DF938C016EE770E08CE589
:102C800094E00E94C901E801F12CF0E2EF2E8E01E0
:102C900088818D57823048F46DE770E08CE594E0D0
:102CA0000E94C90188818E2588832196F801608160
:102CB0008CE594E00E94591FF394F9E0FF12E7CFEE
:102CC0006EE770E08CE594E00E94C901CDB7DEB7F5
:102CD000E6E00C94CA26A9E0B0E0E1E7F6E10C9446
:102CE000B22690915B0391110EC09EEF99838A8367
:102CF0006B8350E0559547954C832D831986188634
:102D00001F821E822EC040916003842F90E0B4E0A9
:102D100095958795BA95E1F7242F2F7030E08217AB
:102D2000930719F18DEF89831B82FE01349650E0E1
:102D3000842F90E0A4E095958795AA95E1F7242F3C
:102D40002F7030E08217930749F0DC01AF59BC4F78
:102D50008C918193405F5F5F563051F740936003E1
:102D60005A83CE0101960E94361680915B0390E053
:102D7000019666E070E00E944D2680935B032996E1
:102D8000E2E00C94CE26A0E0B0E0E9ECF6E10C9491
:102D9000AB266C016EE770E08CE594E00E94C901FF
:102DA0008601E12CF12CC0E0D0E030E2B32EF80136
:102DB000608183E8860F823078F46DE770E08CE5FF
:102DC00094E00E94C901F80160816B2570E08CE5F8
:102DD00094E00E94C90104C08CE594E00E94591F50
:102DE000E114F10459F0F80180819E01280F311D92
:102DF000C901C92FDD27C80FD91FDD273FEFE31A0F
:102E0000F30A89E0E816F10459F028E0E216F1042B
:102E100021F48C2F8095F60180870F5F1F4FC7CF5D
:102E2000CDB7DEB7E9E00C94C726A9E0B0E0EBE14E
:102E3000F7E10C94B226E82F362F80915B0390E0E7
:102E4000019664E270E00E944D2680935B0358E98E
:102E5000598350E15A83813089F048F08230B9F0CB
:102E60008330D9F48B8381EF8C833D8319C085E057
:102E70008B8381EF8C832F5F2D8312C08B8381EF37
:102E80008C8384E6489FA00111245D8309C084E0FF
:102E90008B8381EF8C83ED8303C00E94240904C0DF
:102EA000CE0101960E94C3162996E2E00C94CE262C
:102EB000A2E0B0E0EEE5F7E10C94A726182F762EFD
:102EC0002A8349830E94141B6B017C01809171034A
:102ED00080905C0390905D03A0905E03B0905F03D0
:102EE0002A8149818823C1F0D701C601881999092F
:102EF000AA09BB094C015D0191EE89169EE2990673
:102F0000A104B10420F1241708F4422F202F672DCB
:102F1000812F0E94151713C0D701C601881999097E
:102F2000AA09BB094C015D0191E3891695E7990651
:102F3000A104B10460F0672D812F0E946B16C0922E
:102F40005C03D0925D03E0925E03F0925F032296F1
:102F5000EDE00C94C326A2E2B0E0E1EBF7E10C94C3
:102F6000A8268CE00E941E0581110DC06DE072E064
:102F70008AE094E00E941C1E5F9A80E00E94030693
:102F80000E94DE065F988CE594E00E94FF1E892B6C
:102F900001F18CE594E00E942C1F90913903992354
:102FA00019F00E944A0BEFCF4091CE0250E09A01F7
:102FB0002F5F3F4F2F7133276091CF0270E02617AC
:102FC000370709F3FA01E752FD4F80832093CE02C1
:102FD000DACF80913903811106C080919F0384303C
:102FE00009F094C00DC08AE094E00E94811C892BF6
:102FF000A1F38AE094E00E94A51C0E944A0BF3CF43
:103000000E94141B611571058105910549F06093BB
:103010004B0370934C0380934D0390934E030CC06D
:1030200081E090E0A0E0B0E080934B0390934C03EC
:10303000A0934D03B0934E0380913D0390913E03C6
:10304000816090933E0380933D0383E080939F03D0
:103050008FE70E94FC0409EF12E00E940F05F801BF
:1030600081938F01F3E002301F07B9F7209102032B
:103070008091F902982F922796FF3BC090E4922707
:1030800090930203982F98739833F1F410E0212F56
:1030900030E08091F902877090E0821793074CF13D
:1030A0001F5F2091CA03812F90E0FC01E750FD4F84
:1030B00024FF04C080810E940609E9CF60818CE56D
:1030C00094E00E94591FE3CF8F7399F48091FA0224
:1030D000809346038091FB02809344038091FC021D
:1030E000809343038091FF0290E090933C03809390
:1030F0003B038091CD02813019F482E08093CD02B0
:103100008091CD02833011F41092CD020E94141BE5
:103110006B017C0180913F0390914003A09141039A
:10312000B09142030097A105B105C9F0A70196012E
:10313000281B390B4A0B5B0BDA01C901883B9B400A
:10314000A105B10560F00E944D05809345031092E2
:103150003F0310924003109241031092420380916A
:103160004F0390915003A0915103B0915203460137
:103170005701881A990AAA0ABB0A82EA93E00E94B8
:10318000780386169706A806B90608F4B1C0C0925F
:103190004F03D0925003E0925103F09252030E94E9
:1031A000C00180913A038830A0F08091EB039091A8
:1031B000EC03A091ED03B091EE035CE1B695A79509
:1031C000979587955A95D1F7892B8A2B8B2B09F0E8
:1031D000C4C180913A038F5F80933A0380914B037F
:1031E00090914C03A0914D03B0914E030097A1051F
:1031F000B105F1F0C81AD90AEA0AFB0A82EA93E09B
:103200000E9478036C157D058E059F0508F01BC193
:103210008091EB0384FD04C080ED97E00E94FF02E3
:1032200010924B0310924C0310924D0310924E03D8
:1032300090910203907C909302035091CE02809172
:10324000CF022091CD02581709F41AC1223009F09B
:1032500017C1905890930203E091CA03E770F0E021
:10326000E45EFD4F6081693008F0F2C0615040E0DB
:103270004613F0C08093CF0287E3840F909102033E
:10328000892B809302034093D00283E08093CD0288
:10329000469A1091AF038091590381113EC18091EC
:1032A000EB0382FD46C1812F0E94FE0580915A03E7
:1032B0000E943705E091CA03E770F0E0E45EFD4F3D
:1032C000608182E093E00E9419078091EB0382FD08
:1032D00039C1E0915A03EF5FE0935A03E83109F4F2
:1032E00039C1F0E0EE55FC4F8785882309F432C1DF
:1032F0000E948807813069F58091CA03887149F17D
:1033000080913D0390913E03880F991F90933E0357
:1033100080933D0383E080939F030E94DE060E941A
:10332000141B60933F037093400380934103909379
:103330004203672B682B692B61F481E090E0A0E0E9
:10334000B0E080933F0390934003A0934103B09378
:1033500042038091CA0384FF2BC080914B0390915C
:103360004C03A0914D03B0914E03892B8A2B8B2BDC
:10337000F9F080913D0390913E038E7F0E94AE0450
:10338000182F60913B03809146030E94400B482F09
:10339000612F8091450349A30E94400B00910004D6
:1033A000282F49A160914303809144030E9458173C
:1033B0004698809157038130C1F018F08230B1F106
:1033C000D9C082E10E94581C892B09F0D3C081E04A
:1033D000809357030E94081B609353037093540318
:1033E0008093550390935603C5C082E10E94581CF8
:1033F000892B31F50E94081BC0905303D0905403D1
:10340000E0905503F09056036C197D098E099F09D1
:10341000693E73408105910508F4ACC082E0809359
:10342000570380ED97E00E94FF02A4C082E10E9452
:10343000581C892B09F49EC080E090E00E94FF0296
:103440001092570397C080E090E00E94FF02F0CEF8
:1034500068E00DCF851709F40DCF4F5F242F30E0C2
:1034600090E0F901EE5FFC4FDC01A752BD4F7C916B
:103470007083F901E053FD4F708301968F71F8CE90
:103480002430B1F42091D00281ED92E0A3E0B3E0CA
:10349000FC013E2F381B321718F431913D93F9CFC0
:1034A00087E3820F90910203892B80930203EDCE74
:1034B00080915703823051F49160909302035F9A98
:1034C0008E010F5F1F4FF12CB80110C05F988091E3
:1034D000CD02811103C081E08093CD028091CD02A5
:1034E000833071F784E08093CD02EACF8F2D69A3FA
:1034F0007AA30E94690DF801819391938F01F3944F
:1035000069A17AA1F0E1FF12F1CF8091CA0343E0F3
:1035100053E087700E94FD03BBCE112309F4BFCE98
:103520009091580321E0290F209358039813B7CEA8
:103530001DC082E00E94581C892B09F0B4CE5F9A0E
:1035400017E0B1CE82E00E94581C892B09F0C1CE51
:103550005F98BFCE10925A03CBCE80913A03883049
:1035600009F45F9A89E080933A03C2CE109258031F
:10357000115095CEA296ECE00C94C4261F920F92A7
:103580000FB60F9211242F933F938F939F93AF9376
:10359000BF938091020490910304A0910404B09120
:1035A00005043091010423E0230F2D3720F4019608
:1035B000A11DB11D05C026E8230F0296A11DB11D56
:1035C000209301048093020490930304A0930404C5
:1035D000B09305048091060490910704A09108041B
:1035E000B09109040196A11DB11D8093060490932A
:1035F0000704A0930804B0930904BF91AF919F9171
:103600008F913F912F910F900FBE0F901F901895A3
:103610002FB7F89460910204709103048091040420
:10362000909105042FBF08953FB7F8948091060448
:1036300090910704A0910804B091090426B5A89BB5
:1036400005C02F3F19F00196A11DB11D3FBF662790
:10365000782F892F9A2F620F711D811D911D42E0D5
:10366000660F771F881F991F4A95D1F70895CF924B
:10367000DF92EF92FF92CF93DF936B017C010E9468
:10368000141BEB01C114D104E104F10479F00E9490
:10369000141B6C1B7D0B683E7340A0F381E0C81ABD
:1036A000D108E108F108C851DC4FECCFDF91CF9190
:1036B000FF90EF90DF90CF900895789484B582606A
:1036C00084BD84B5816084BD85B5826085BD85B5C6
:1036D000816085BDEEE6F0E0808181608083E1E875
:1036E000F0E01082808182608083808181608083AD
:1036F000E0E8F0E0808181608083E1E9F0E08081B2
:1037000082608083808181608083E0E9F0E0808155
:1037100081608083E1ECF0E080818460808380813F
:1037200082608083808181608083E3ECF0E080812F
:1037300081608083E0ECF0E0808182608083E2EC55
:10374000F0E0808181608083EAE7F0E0808184603E
:10375000808380818260808380818160808380819A
:1037600080688083089590E0FC013197EE30F10588
:1037700090F5E35AFF4F0C94D926809180008F7703
:1037800003C0809180008F7D80938000089584B570
:103790008F7702C084B58F7D84BD0895809190009D
:1037A0008F7707C0809190008F7D03C0809190003B
:1037B000877F8093900008958091C0008F7703C029
:1037C0008091C0008F7D8093C00008958091C200D9
:1037D000877F8093C2000895CF93DF9390E0FC0130
:1037E000E75EFE4F2491FC01E95CFE4F8491882343
:1037F00049F190E0880F991FFC01EF58FE4FA59109
:10380000B4918D599E4FFC01C591D4919FB7611120
:1038100008C0F8948C91209582238C938881822310
:103820000AC0623051F4F8948C91322F3095832382
:103830008C938881822B888304C0F8948C91822B8E
:103840008C939FBFDF91CF910895A1E0B0E0EBE2B0
:10385000FCE10C94B026282F30E0F901E550FF4F31
:103860008491F901E75EFE4F1491F901E95CFE4F86
:1038700004910023C9F0882321F069830E94B31BBF
:103880006981E02FF0E0EE0FFF1FED59FE4FA5918B
:10389000B4919FB7F8948C91611103C01095812366
:1038A00001C0812B8C939FBF2196E4E00C94CC2621
:1038B000CF93DF93282F30E0F901E550FF4F84913B
:1038C000F901E75EFE4FD491F901E95CFE4FC49126
:1038D000CC2391F081110E94B31BEC2FF0E0EE0F8E
:1038E000FF1FEB5AFE4FA591B4912C912D2381E03F
:1038F00090E021F480E002C080E090E0DF91CF9181
:103900000895809158049091590420915A0430915F
:103910005B04821B930B8F739927089520915804A1
:103920003091590480915A0490915B04281739070B
:1039300049F0E0915A04F0915B04E85EFB4F80810E
:1039400090E008958FEF9FEF0895209158043091F3
:10395000590480915A0490915B0428173907A9F003
:10396000E0915A04F0915B04E85EFB4F8081209166
:103970005A0430915B042F5F3F4F2F7333273093EE
:103980005B0420935A0490E008958FEF9FEF089511
:10399000CF93DF93C0915804D09159042196CF73EF
:1039A000DD2780915A0490915B04C817D90799F0DC
:1039B00082E00E9403228F3F2FEF920761F0E09197
:1039C0005804F0915904E85EFB4F8083D09359046A
:1039D000C0935804DFCFDF91CF91089583E00E9418
:1039E0004E240895A1E0B0E0E8EFFCE10C94B0268D
:1039F0008C0169838091A401882359F041E050E053
:103A0000BE016F5F7F4F83E00E94362218161906B1
:103A10003CF081E090E0F8019383828380E090E0C5
:103A20002196E4E00C94CC26FC0120812E5F2083BB
:103A300042E450E06FE771E080E80E94B62208950A
:103A4000FC0181819081913A59F4813209F04BC097
:103A500047E050E06DE971E080E00E94B62245C089
:103A6000913209F040C0803239F467E070E08DE9AE
:103A700091E00E94FA2239C0823209F034C082817A
:103A80008093A40180919D0190919E01A0919F013E
:103A9000B091A001803B9440A105B10531F5809122
:103AA000A40180FD12C087E797E7909301088093F7
:103AB00000082BE088E190E00FB6F894A895809379
:103AC00060000FBE2093600010C088E10FB6F8942C
:103AD00080936000109260000FBEA89510920108BC
:103AE0001092000802C080E0089581E008950895D2
:103AF00010920D0410920C0488EE93E0A0E0B0E068
:103B000080930E0490930F04A0931004B0931104BB
:103B10008EE292E090930B0480930A040895A0E053
:103B2000B0E0E5E9FDE10C94AC266C017A01EB0113
:103B3000E60EF71E00E010E0CE15DF0561F069919A
:103B4000D601ED91FC910190F081E02DC60109951F
:103B5000080F191FF1CFC801CDB7DEB7E8E00C940C
:103B6000C8266115710589F0DB010D900020E9F789
:103B7000AD0141505109461B570BDC01ED91FC9101
:103B80000280F381E02D0995089580E090E008958A
:103B9000EF92FF920F931F93CF93DF938C01FB0162
:103BA000C0E0D0E064917F018FEFE81AF80A662345
:103BB00061F0D801ED91FC910190F081E02DC801F8
:103BC0000995C80FD91FF701EDCFCE01CDB7DEB7EC
:103BD000E6E00C94CA260E94B11D0895DC01ED9127
:103BE000FC910190F081E02D099508950F931F93AA
:103BF000CF93DF93EC016DE00E94EE1D8C016AE033
:103C0000CE010E94EE1D800F911FDF91CF911F9179
:103C10000F9108950F931F93CF93DF93EC010E94B0
:103C2000C81D8C01CE010E94F61D800F911FDF91EF
:103C3000CF911F910F9108950F931F93CF93DF930F
:103C4000EC010E94B11D8C01CE010E94F61D800F77
:103C5000911FDF91CF911F910F9108950F931F93A3
:103C6000CF93DF93EC010E94EE1D8C01CE010E94E8
:103C7000F61D800F911FDF91CF911F910F91089535
:103C8000A1E2B0E0E6E4FEE10C94A8267C01C42E9B
:103C9000E52FCB01D22E19A221E02D1510F02AE03C
:103CA000D22E8E010F5D1F4F8D2C912CA12CB12C8B
:103CB0006C2D7E2FA50194010E9461268C2DD29E31
:103CC00080191124015011098A3010F4805D01C05F
:103CD000895CF8018083211531054105510521F0EA
:103CE000C22EE32FCA01E4CFB801C7010E94B11D63
:103CF000A196ECE00C94C426A0E0B0E0E2E8FEE17E
:103D00000C94AC26EC016A017B012115310541F4CC
:103D1000E881F9810190F081E02D642F09951DC0A3
:103D20002A303105A9F477FF12C06DE20E94EE1D22
:103D30008C0144275527BA014C195D096E097F098A
:103D40002AE0CE010E94401E800F911F06C02AE08B
:103D5000B701A601CE010E94401ECDB7DEB7E8E054
:103D60000C94C8260F931F93CF93DF93EC019A0115
:103D7000AB01662757FD6095762F0E947C1E8C0153
:103D8000CE010E94F61D800F911FDF91CF911F91F0
:103D90000F9108952115310549F4DC01ED91FC9155
:103DA0000190F081E02D642F099508950E94401E36
:103DB00008959A01462F50E060E070E00E94CA1E0C
:103DC00008959A01AB0160E070E00E94CA1E089558
:103DD0000F931F93CF93DF93EC019A01462F50E08E
:103DE00060E070E00E94CA1E8C01CE010E94F61DA8
:103DF000800F911FDF91CF911F910F910895FC01CA
:103E000024853585F901E05CFF4F80819181F901BE
:103E1000EE5BFF4F20813181821B930B8F739927BB
:103E20000895FC0184859585FC01E05CFF4F40818D
:103E30005181FC01EE5BFF4F208131814217530716
:103E400041F00190F081E02DE80FF91F808190E0B2
:103E500008958FEF9FEF0895FC0184859585FC01FF
:103E6000E05CFF4F40815181FC01EE5BFF4F208100
:103E700031814217530779F0A081B181A80FB91F92
:103E80008C91208131812F5F3F4F2F7333273183F6
:103E9000208390E008958FEF9FEF0895FC0181A1AA
:103EA000882329F0A489B5898C9186FFFBCF11A2C4
:103EB0000895CF93DF93FC0126853785D901A05C57
:103EC000BF4F8D919C91119701968F739927E901AE
:103ED000CE5BDF4F4881598184179507D9F30D9048
:103EE000BC91A02DA20FB31F6C93A685B785A05CD3
:103EF000BF4F11969C938E93A689B7892C9181E030
:103F000090E0078C02C0880F991F0A94E2F7282BD3
:103F10002C9381E081A30488F589E02D8081806461
:103F2000808381E090E0DF91CF91089508951F9202
:103F30000F920FB60F9211242F933F934F938F93AD
:103F40009F93EF93FF938091C80082FD1CC0409126
:103F5000CE00809102059091030501968F739927F9
:103F600020910405309105058217930771F0E091C7
:103F70000205F0910305EE53FB4F40839093030538
:103F80008093020502C08091CE00FF91EF919F9136
:103F90008F914F913F912F910F900FBE0F901F90D7
:103FA00018958CE594E00E94FF1E892B11F00E9469
:103FB000961F08951F920F920FB60F9211242F9300
:103FC0003F938F939F93EF93FF932091BE04309183
:103FD000BF048091C0049091C1042817390731F4BF
:103FE0008091C9008F7D8093C90014C0E091C00406
:103FF000F091C104E258FB4F20818091C004909160
:10400000C10401968F7399279093C1048093C004D3
:104010002093CE00FF91EF919F918F913F912F912F
:104020000F900FBE0F901F901895A0E0B0E0EBE14D
:10403000F0E20C94A826FC011382128288EE93E031
:10404000A0E0B0E084839583A683B78380E492E008
:10405000918380837587648757874687318B208B50
:10406000138B028BF58AE48AD78AC68AB18EA08E1A
:10407000938E828E8F85848F8889858F8989868F9C
:104080008A89878F8B8980A3ECE00C94C426CF9219
:10409000DF92EF92FF92CF93DF93EC016A017B01F5
:1040A000411581EE580761057105F9F0EC89FD892C
:1040B00081E090E008A002C0880F991F0A94E2F7FF
:1040C000808360E079E08DE390E0A70196010E9493
:1040D0006126215031094109510956954795379577
:1040E0002795211580E1380798F0EC89FD89108229
:1040F00060E874E88EE190E0A70196010E946126D5
:104100002150310941095109569547953795279511
:10411000E889F9893083EA89FB89208319A2EE892D
:10412000FF89408181E090E09C010C8C02C0220F4D
:10413000331F0A94E2F7422B4083EE89FF894081C6
:104140009C010D8C02C0220F331F0A94E2F7422B10
:104150004083EE89FF8940819C010E8C02C0220FB2
:10416000331F0A94E2F7422B4083EE89FF892081B6
:104170000F8C02C0880F991F0A94E2F78095822362
:104180008083DF91CF91FF90EF90DF90CF900895E3
:10419000BF92CF92DF92EF92FF92CF93DF93EC0129
:1041A0006A017B01B22E411581EE58076105710548
:1041B000F9F0EC89FD8981E090E008A002C0880F49
:1041C000991F0A94E2F7808360E079E08DE390E044
:1041D000A70196010E946126215031094109510928
:1041E0005695479537952795211580E1380798F022
:1041F000EC89FD89108260E874E88EE190E0A70107
:1042000096010E94612621503109410951095695B4
:10421000479537952795E889F9893083EA89FB899D
:104220002083E88DF98DB082EE89FF89408181E09D
:1042300090E09C010C8C02C0220F331F0A94E2F71D
:10424000422B4083EE89FF8940819C010D8C02C086
:10425000220F331F0A94E2F7422B4083EE89FF8935
:1042600040819C010E8C02C0220F331F0A94E2F79A
:10427000422B4083EE89FF8920810F8C02C0880F7A
:10428000991F0A94E2F7809582238083DF91CF9172
:10429000FF90EF90DF90CF90BF9008958F929F9204
:1042A000AF92BF92CF92DF92EF92FF920F931F9344
:1042B00081E08F9385E08F9387E08F9383E08F93E6
:1042C00084E08F93EEEC8E2E912CFAECAF2EB12C75
:1042D000A9ECCA2ED12CB8ECEB2EF12C0CEC10E092
:1042E0002DEC30E04EE754E062EC74E08CE594E0B5
:1042F0000E9415200F900F900F900F900F901F911C
:104300000F91FF90EF90DF90CF90BF90AF909F9074
:104310008F9008950E945D1B86E095E00E945824CE
:104320000E940415C1EDDFE10E94AB172097E1F375
:104330000E94D11FF9CF615030F02091F100FC01B3
:1043400020830196F8CF289884E680930D05089580
:104350002FB7FC012083F89467706093E9000895FB
:10436000A1E0B0E0E6EBF1E20C94B226682FCE01BA
:1043700001960E94A8218091F20099819FBF219609
:10438000E2E00C94CE26A2E0B0E0E9ECF1E20C947D
:10439000AF26F62E8A0190910C05992311F057FF54
:1043A00003C08FEF9FEF2BC0682FCE0101967A8359
:1043B0000E94A8218091F20090E0A8017A818017E4
:1043C00091070CF4AC01EF2DF72FF40E84E6FE16E6
:1043D00039F0289880930D059091F1009193F7CFD3
:1043E0004115510521F08091F200882321F0898147
:1043F0008FBFCA0104C08BE68093E800F8CF2296F5
:10440000E5E00C94CB26A1E0B0E0E9E0F2E20C9408
:10441000B22641E050E0BE016F5F7F4F0E94C32192
:10442000019719F4898190E002C08FEF9FEF2196E8
:10443000E2E00C94CE26A1E0B0E0E1E2F2E20C94DE
:10444000B226682FCE0101960E94A8219091E80023
:10445000892F807295FF04C09091F20080E4891B3F
:1044600099819FBF2196E2E00C94CE26A1E0B0E0B6
:10447000ECE3F2E20C94A426582E7B01A42E952E98
:1044800080910C05882369F0042F152F8AEFB82E30
:10449000852D8072782E9AE3892E852D8074682E62
:1044A00011C08FEF9FEF53C0852D0E941B22482E15
:1044B00081110CC0BA94A9F361E070E080E090E053
:1044C0000E94371B0115110579F737C0282F30E0FE
:1044D000021713070CF4402EC42CD12C0C191D0903
:1044E000652DCE0101960E94A821772039F04A94CB
:1044F0008FEF4816B1F01092F100F9CFF701842D3B
:1045000057FE07C0815058F094919093F100319676
:10451000F9CF815020F091919093F100FACFEC0CFB
:10452000FD1C8091E80085FF0FC00115110511F4F5
:1045300061100AC089818FBFC5CF5D9884E68093E2
:104540000E058A2D992D03C08092E800F3CF2196A5
:10455000E0E10C94C0261092E90010920B05109235
:104560000A0590930905809308050895CF93DF937A
:10457000FB0120E030E0DEEF24173507A1F187FFD3
:1045800002C0C49101C0C081A0910A05B0910B0581
:104590006091080570910905A617B707B4F49091CA
:1045A000E8009570E1F39091E80092FD1EC0C09381
:1045B000F10060910A0570910B056F5F7F4F6F737B
:1045C0007727672B11F4D093E80060910A0570916A
:1045D0000B056F5F7F4F70930B0560930A052F5F8C
:1045E0003F4F3196C9CFC90102C08FEF9FEFDF91D6
:1045F000CF910895A1E0B0E0E0E0F3E20C94B126A1
:10460000162F2091E80022FFFCCF612F79830E94B2
:104610009B218BEF8093E800812F7981972F219642
:10462000E3E00C94CD26A1E0B0E0E9E1F3E20C94E4
:10463000B2261982CE0101960E94141DCE01019668
:104640000E94F224898190E02196E2E00C94CE262B
:104650001F920F920FB60F921124EF92FF920F93B9
:104660001F932F933F934F935F936F937F938F93FA
:104670009F93AF93BF93EF93FF93CF93DF93CDB708
:10468000DEB76297DEBFCDBF1092E9008091E800EF
:1046900083FFE7C068E0CE010A960E949B2182EF6B
:1046A0008093E8009A8597FF05C08091E80080FF1D
:1046B000FCCF03C08EEF8093E800892F807609F04D
:1046C000B5C08B85811105C01092F1001092F100E8
:1046D000C1C0282F2D7F213009F4BCC0853049F49A
:1046E0008091E80080FFFCCF8C8580688093E30098
:1046F000B1C0863009F072C02D85E888F988223073
:1047000071F580E090E02A8B0E94AB220E94132377
:1047100099E08E010F5F1F4FF801392F11923A95E2
:10472000E9F799832A892A8391E09E8390E8988704
:104730009AEF998720910A0530910B05275F3F4F2B
:104740003C832B838D83C7010E94AB2249E050E05C
:10475000B80180E00E94B6220E9413237BC0C701EB
:104760002A8B0E94AB222A89223241F482E290E015
:104770000E94FE24892B09F06DC070C0213069F4BD
:1047800088899989089711F4209307058091070576
:10479000882389F066EC71E016C0233009F05EC012
:1047A0008C85882359F0823061F0813009F056C041
:1047B0006AEE71E008C068ED71E005C064E272E085
:1047C00002C062E072E06115710509F447C0FB01A7
:1047D000449150E080E80E94B6223CC0873009F442
:1047E0003DC0883021F481E08093F10033C08930EE
:1047F00089F5937099F5E2ECF1E081E021E096E330
:104800008093E9002093EB0034913093EC00909377
:10481000ED008F5F3196853099F78EE78093EA003F
:104820001092EA008C8580930C0514C088899989C0
:104830000E94AB228E85811105C0CE010A960E948E
:10484000201D06C0823051F4CE010A960E94202518
:10485000882321F08EEF8093E80003C081E28093EB
:10486000EB0062960FB6F894DEBF0FBECDBFDF91AE
:10487000CF91FF91EF91BF91AF919F918F917F91D8
:104880006F915F914F913F912F911F910F91FF90E9
:10489000EF900F900FBE0F901F9018958093E90036
:1048A0008091F200882319F08AE38093E80008954C
:1048B00010920C0581E08093D70080EA8093D800A5
:1048C00082E189BD09B400FEFDCF61E070E080E0C7
:1048D00090E00E94371B80E98093D8008CE08093A1
:1048E000E2001092E000559A209A08951F920F92CC
:1048F0000FB60F9211242F933F934F935F936F93B3
:104900007F938F939F93AF93BF93EF93FF93809188
:10491000E1001092E10083FF0FC01092E90091E0E6
:104920009093EB001092EC0092E39093ED001092C4
:104930000C0598E09093F00082FF26C083E00E946F
:104940004E2482E00E94B021882321F08AE094E086
:104950000E94C81C80910E05882339F080910E05B5
:10496000815080930E05882369F080910D0588237E
:1049700059F080910D05815080930D05811104C07F
:10498000289A02C05D9AF1CFFF91EF91BF91AF914C
:104990009F918F917F916F915F914F913F912F9157
:1049A0000F900FBE0F901F901895FF920F931F93BB
:1049B000CF93DF93EC01F62EE881F9810480F58135
:1049C000E02D09958C01E881F9810680F781E02DC1
:1049D0006F2DCE010995C8019927CDB7DEB7E5E067
:1049E0000C94CB26FC0120812F5F208349E150E00D
:1049F00068EA72E080E80E94B622089545E650E039
:104A000061EC72E080E80E94B6220895A1E0B0E077
:104A1000ECE0F5E20C94AE2689838B017A0141E04B
:104A200050E0BE016F5F7F4F84E00E943622A701F5
:104A3000B80184E40E9436222196E6E00C94CA264E
:104A4000FC0191818081813A31F481E0913091F0D3
:104A5000933089F411C0813271F49B3021F482814A
:104A60008093A60105C09A3031F482818093A5011C
:104A700081E00895089580E00895FC011082089572
:104A8000FC011382128220E532E0318320830895F5
:104A900048E050E082E00E9406250895CF93DF931E
:104AA000DC01683818F0E8E7E60F25C0E62FF0E0F3
:104AB00067FF11C0E058F10981E090E001C0880F64
:104AC000EA95EAF714969C911497982B14969C9368
:104AD0001497E0E010C0E85DFD4FE491EE2309F487
:104AE00040C0E7FF08C014968C911497826014961A
:104AF0008C931497EF7716968C9116978E1741F139
:104B000017968C9117978E1719F118968C91189704
:104B10008E17F1F019968C9119978E17C9F01A9685
:104B20008C911A978E17A1F01B968C911B978E175C
:104B300079F080E090E0ED01C80FD91F2E8121119E
:104B400002C0EE8305C0019686309105A1F709C029
:104B5000BD016C5F7F4FCD010E94482581E090E050
:104B600008C081E090E013969C938E93129780E0AA
:104B700090E0DF91CF910895683818F0E8E7E60FEC
:104B800025C0E62FF0E067FF12C0E058F10921E0F0
:104B900030E001C0220FEA95EAF72095DC01149677
:104BA0003C911497322314963C93E0E00FC0E85DEB
:104BB000FD4FE491EE2329F1E7FF08C0DC011496D4
:104BC0002C9114972D7F14962C93EF7720E030E0F2
:104BD000EE2351F0DC01A20FB31F16964C911697ED
:104BE0004E1302C016961C922F5F3F4F26303105A0
:104BF00079F7BC016C5F7F4F0E94482581E090E00F
:104C0000089580E090E00895FC01168217821086D6
:104C10001186128613861482BC016C5F7F4F0E943E
:104C2000482508958BE195E00E943D258FE095E0B1
:104C30000E9440250895A29FB001B39FC001A39F89
:104C4000700D811D1124911DB29F700D811D1124C5
:104C5000911D08950E941B26A59F900DB49F900D55
:104C6000A49F800D911D11240895B7FF0C942A264E
:104C70000E942A26821B930B0895DB018F939F933A
:104C80000E942A26BF91AF91A29F800D911DA39FE4
:104C9000900DB29F900D1124089597FB072E16F4E6
:104CA000009407D077FD09D00E94DF2607FC05D0CD
:104CB0003EF4909581959F4F0895709561957F4F33
:104CC0000895A1E21A2EAA1BBB1BFD010DC0AA1F4D
:104CD000BB1FEE1FFF1FA217B307E407F50720F065
:104CE000A21BB30BE40BF50B661F771F881F991FE0
:104CF0001A9469F760957095809590959B01AC0129
:104D0000BD01CF010895052E97FB1EF400940E946B
:104D10009A2657FD07D00E94612607FC03D04EF467
:104D20000C949A2650954095309521953F4F4F4FC2
:104D30005F4F089590958095709561957F4F8F4F47
:104D40009F4F08952F923F924F925F926F927F9262
:104D50008F929F92AF92BF92CF92DF92EF92FF928B
:104D60000F931F93CF93DF93CDB7DEB7CA1BDB0B37
:104D70000FB6F894DEBF0FBECDBF09942A883988DC
:104D800048885F846E847D848C849B84AA84B984E3
:104D9000C884DF80EE80FD800C811B81AA81B981EF
:104DA000CE0FD11D0FB6F894DEBF0FBECDBFED0103
:104DB0000895EE0FFF1F0590F491E02D0994AA1BB2
:104DC000BB1B51E107C0AA1FBB1FA617B70710F0F6
:104DD000A61BB70B881F991F5A95A9F78095909528
:104DE000BC01CD0108958F929F92AF92BF92CF9256
:104DF000DF92EF92FF92CF93DF93EC01688179818C
:104E00008A819B81611571058105910521F464E218
:104E100079ED8BE597E02DE133EF41E050E00E9422
:104E2000832649015A019B01AC01A7EAB1E40E9423
:104E30002A266B017C01ACEEB4EFA50194010E941F
:104E40003826C60ED71EE81EF91EF7FE06C081E002
:104E5000C81AD108E10880E8F80AC882D982EA8233
:104E6000FB82C701B6019F77DF91CF91FF90EF9052
:104E7000DF90CF90BF90AF909F908F9008950E9449
:104E8000F326089586E091E00E94F326089560934A
:104E9000060170930701809308019093090108951A
:104EA000F999FECF92BD81BDF89A992780B50895F2
:104EB000262FF999FECF1FBA92BD81BD20BD0FB636
:104EC000F894FA9AF99A0FBE01960895F894FFCFD4
:104ED00000001C05200001000000FF00020002008D
:104EE00002000200020002000200020002000200B2
:104EF00002000200020002000200028025000005FC
:104F0000400AA1204EA50020244EA52C2330C0121B
:104F100000001A400AA1204EA5001B1E27522C2378
:104F2000308025000005400AA1204EA50020244E17
:104F3000A52C2330004B000006400AD0009D4900FC
:104F40007B289D492C233000E1000005400A4501E3
:104F5000D7DC03B81E0EBF00232E48E801008A40AC
:104F60000A6001555502AD1E20000023C800E10073
:104F70000000000000010154582074696D656F75D0
:104F8000742100456E746572696E6720616461709A
:104F900074697665206368616E6E656C2073656CFC
:104FA000656374696F6E2C207069636B696E673A14
:104FB000007363616E6E6572206D6F6465004F7083
:104FC000656E4C52536E672054582073746172742E
:104FD000696E672000206F6E20485720006D6F6457
:104FE000756C65206C6F636B65643F0000070B0C8C
:104FF00010111500160A1322312900000000F21CBE
:105000008F1D811CA51C8E1CEE1CC81C00000000FE
:10501000591F8F1DFF1E2C1F111F4E1F0000000067
:0A502000D5248F1D4E25BC25042663
:00000001FF
